:10000000B40149299818181218162C08A0002D08B8
:10001000A100A201A3010C280D2864008C1A292834
:10002000FF30A207031CA307031CA007031CA107A2
:10003000031C4429220F0B28230F0C28FA30A2009E
:100040000030A3000D2898181812181664008C1E92
:1000500026281A0803144429B416B41EB4123419FD
:100060003628FE39B500341503104429341A3E28C9
:10007000A600341655200318432826085C200318D0
:100080004328B41E44294E20732034113412B41175
:1000900038088400360884178004542838088400FF
:1000A00036098005841780050800482073204E20FB
:1000B0006F203508B4190138A2000830A300A20D42
:1000C00003184820031C4E2073206F20A30B5F28C9
:1000D000482073203808840036080005FF3E3908A0
:1000E0008400370951283908840037084B28B600A6
:1000F000E12020082104031944293E2184133608F5
:100100008006640083288428A00A0319A10F81288F
:10011000800644290830A600A70039088400370863
:100120003519D920351DDB20380884003608DE203B
:10013000A001A101260803194429B518CE203808CA
:10014000840000083605FF3EA00DA10DB51CCE2091
:10015000A60B9D28270835180929200844290830AE
:10016000A6003908840037083519D920351DDB2051
:10017000380884003609E220260803194429351876
:10018000092138088400A10CA00C00083604031CC7
:1001900036068000CE20A60BC128442939088400E9
:1001A000370880060000D428D528D628D72880060E
:1001B00008008004E128FF3A8005E22884178004C3
:1001C0004429FF3A84178005442983178001840A53
:1001D000FF3E031DE6284429A301A200FF30A20729
:1001E000031CA307031C44290330A100E630FA20B6
:1001F000EE28A101FC3EA000A109031C0529FF3047
:100200000000A00703180029A0076400A10FFF2821
:100210000800A201A3011029A10CA00CA20DA30D9E
:10022000FF3E03180C292308A1002208A00044293E
:100230000310A00DA10DFF3E031818292008442922
:100240000310A10CA00CFF3E03182029200844290C
:100250001030A800A101A001A70CA60C031C362990
:100260002208A00723080318230FA107A10CA00C44
:10027000A50CA40CA80B2C2924084429A009A10929
:10028000A00A0319A10A0800831303138312640050
:1002900008008316043099002430980083129030AF
:1002A000980007309F0083163C308500023086009E
:1002B0002030840060308312E620A030840050306B
:1002C000E620203084003030E5200617861706141B
:1002D00005140A30F92085140A30F92085100A30F7
:1002E000F92005101930F9200530B8000430B600A7
:1002F0000530B9000230B7000130B5008A20EC00AB
:100300006430F92038300505ED006D08A000A1012A
:1003100003302321EE00640003306E02031C912998
:10032000B129851406100A30F9200530B8000130D3
:10033000B6000530B9000230B7000130B5006C08D6
:10034000A000A101AF200A30F92006140A30F920DC
:1003500006100A30F920061485100130A100F4308F
:10036000FA2086110130AC00AD010220031CB12936
:10037000243C031DB5290220031CB129EB006400B5
:100380006B08003C031DC529C629B129EF01640093
:1003900021306F020318D5292320EB006F083A3E65
:1003A00084006B088000EF0FC72964006E08003CD2
:1003B000031DDC290D220C2A64006E08013C031D7C
:1003C000E32949220C2A64006E08023C031DEA2935
:1003D000C4220C2A64006E08033C031DF129022389
:1003E0000C2A64006E08043C031DF82923230C2A00
:1003F00064006E08053C031DFF2980230C2A64005D
:100400006E08063C031D062AB1290C2A64006E08FA
:10041000073C031D0C2AB129B1290617EF0164001E
:1004200004306F020318482A6F08A600A7010430A1
:10043000A200A3012821B2002508B3000230320730
:10044000E6006F086C07B200B301B30D32083A3E04
:1004500084000008E5006508A0006608A1000430DB
:100460001B21E7002108E80006130630B800103011
:10047000B6000630B9002030B7000530B500670877
:10048000A0006808A1001030B0200617EF0F0F2A57
:1004900008000617EF01640004306F020318842A75
:1004A0006F08A600A7010430A200A3012821B20012
:1004B0002508B30002303207E6006F086C07B2006F
:1004C000B301B30D32083A3E84000008E500650828
:1004D000A0006608A10004301B21E7002108E80005
:1004E00006130630B8001030B6000630B9002030D0
:1004F000B7000530B5006708A0006808A1001030FB
:10050000B0200617EF0F4B2A8617EF016400043066
:100510006F020318C32A6F08A600A7010430A200C7
:10052000A3012821B2002508B30002303207E600FB
:100530006F086C07B200B301B30D0430B2070318A3
:10054000B30A32083A3E84000008E5006508A000BE
:100550006608A10004301B21E7002108E80086138B
:100560000630B8001030B6000630B9002030B700B1
:100570000530B5006708A0006808A1001030B02061
:100580008617EF0F862A0800EF01640008306F021B
:100590000318E32A6F086C07B200B301B30D3208E9
:1005A0003A3E84000008B2003208A000A1010230E7
:1005B0002321B2002108B3006F085D3E8400320899
:1005C0008000EF0FC52A0630B8001030B6000630A4
:1005D000B9002030B70040302E2000302E205D08BA
:1005E0002E205E082E205F082E2060082E20610835
:1005F0002E2062082E2063082E2064082C20023052
:10060000EC200800061386120A30F9200630B800E4
:100610001030B6000630B9002030B7000130B50008
:100620006C083A3E84000008B2003208A000A10124
:10063000AF200A30F92006170A30F9200613861277
:100640000A30F920080086120A30F92006138613B2
:1006500006106C08EF0060230617861306106C0A5C
:10066000EF00602306138617061002306C07EF00B8
:10067000602306178617061003306C07EF0060230F
:1006800006138613061404306C07EF006023061768
:100690008613061405306C07EF00602306138617D7
:1006A000061406306C07EF00602306178617061441
:1006B00007306C07EF00602386160A30F920080027
:1006C0006F083A3E84000008B2000230A600A7017D
:1006D0003208A200A3012821B2002508B300F4309B
:1006E0003207E90001300318013E3307EA006908C8
:1006F000A0006A08A10006308400103077200800AE
:1007000064007108003C031D862BF20100306C0769
:10071000B200B301B30D32083A3E84000008B200C3
:10072000640071083202031D962B721401306C07AD
:10073000B200B301B30D32083A3E84000008B200A3
:10074000640071083202031DA62BF21402306C07FC
:10075000B200B301B30D32083A3E84000008B20083
:10076000640071083202031DB62B721503306C074A
:10077000B200B301B30D32083A3E84000008B20063
:10078000640071083202031DC62BF21504306C0799
:10079000B200B301B30D32083A3E84000008B20043
:1007A000640071083202031DD62B721605306C07E7
:1007B000B200B301B30D32083A3E84000008B20023
:1007C000640071083202031DE62BF21606306C0736
:1007D000B200B301B30D32083A3E84000008B20003
:1007E000640071083202031DF62B721707306C0784
:1007F000B200B301B30D32083A3E84000008B200E3
:10080000640071083202031D062CF2177209F3000E
:10081000061386120A30F9200630B8001030B600F0
:100820000630B9002030B7000130B5007308A000D1
:10083000A101AF200A30F92006170A30F92006136B
:1008400086120A30F920F10A64007108003C03198D
:060850002A2C802B080099
:02400E000603A7
:00000001FF
